:020000040000FA
:02000000B02826
:080008008B138B1B04289200EE
:10001000030E930083010A0894008A0183130408E5
:100020009500051A2C2808309600061C152806187D
:100030001728051E1D2898171E289813160B980CB4
:10004000960B152802309600061C24280618262830
:10005000960B2428051A2E2898013C288316031392
:100060000610831203130610180867208316031363
:100070000614831203138B101508840014088A00D9
:0A008000130E8300920E120E090009
:1000A0008C00810183160313C030810508008C0089
:1000B000810183160313C03081050130810483124E
:1000C00003130B110B1D62288C0B61280800900094
:1000D000051008308C00782010180514101C05102D
:1000E000900C78208C0B6C28051478207820080060
:1000F0000C308D007E2801308D007E288D0B7E28EF
:06010000080091013B28FC
:1001600083160313810106140516831203138316E5
:1001700003130510061401138312031305148B10C7
:100180000B168B170530572027308E0000308A0061
:100190000E08273CD32067208E0BC628FF30502046
:1001A00007305E20C4288207503449344334203459
:1001B0003134363446343834343420344B346534B6
:1001C000793462346F3461347234643420344434AA
:1001D000653463346F34643465347234203463348A
:1001E0006F346E346E34653463347434653464341F
:0601F0000D340A340A344C
:02400E00F13F80
:00000001FF
